
 Start  Stop   Length Name                   Class
 00000H 087D3H 087D4H _TEXT                  CODE
 087E0H 0AD0FH 02530H EMULATOR_TEXT          CODE
 0AD10H 0AD10H 00000H C_ETEXT                ENDCODE
 0AD10H 0B50FH 00800H _DATA                  
 0B510H 0B598H 00089H DOSXXX                 DOS
 0B599H 0B6F6H 0015EH VIOXXX                 VIO
 0B700H 0B86FH 00170H EMULATOR_DATA          FAR_DATA
 0B870H 0B8B1H 00042H NULL                   BEGDATA
 0B8B2H 0F7A6H 03EF5H _DATA                  DATA
 0F7A8H 0F7B5H 0000EH CDATA                  DATA
 0F7B6H 0F7B6H 00000H XIFB                   DATA
 0F7B6H 0F7B6H 00000H XIF                    DATA
 0F7B6H 0F7B6H 00000H XIFE                   DATA
 0F7B6H 0F7B6H 00000H XIB                    DATA
 0F7B6H 0F7B7H 00002H XI                     DATA
 0F7B8H 0F7B8H 00000H XIE                    DATA
 0F7B8H 0F7B8H 00000H XPB                    DATA
 0F7B8H 0F7B9H 00002H XP                     DATA
 0F7BAH 0F7BAH 00000H XPE                    DATA
 0F7BAH 0F7BAH 00000H XCB                    DATA
 0F7BAH 0F7BAH 00000H XC                     DATA
 0F7BAH 0F7BAH 00000H XCE                    DATA
 0F7BAH 0F7BAH 00000H XCFB                   DATA
 0F7BAH 0F7BAH 00000H XCF                    DATA
 0F7BAH 0F7BAH 00000H XCFE                   DATA
 0F7BAH 0F7C9H 00010H CONST                  CONST
 0F7CAH 0F7D1H 00008H HDR                    MSG
 0F7D2H 0F976H 001A5H MSG                    MSG
 0F977H 0F978H 00002H PAD                    MSG
 0F979H 0F979H 00001H EPAD                   MSG
 0F97AH 0F9A9H 00030H _BSS                   BSS
 0F9AAH 0F9AAH 00000H XOB                    BSS
 0F9AAH 0F9AAH 00000H XO                     BSS
 0F9AAH 0F9AAH 00000H XOE                    BSS
 0F9B0H 111E5H 01836H c_common               BSS
 111F0H 119EFH 00800H STACK                  STACK

 Origin   Group
 0B87:0   DGROUP

  Address         Publics by Name

 0B87:3E90       $i8_implicit_exp
 0B87:3E8E       $i8_inpbas
 0000:7AE1       $i8_input
 0B87:3E8F       $i8_input_ws
 0000:7F35       $i8_output
 0000:81F6       $i8_tpwr10
 0B87:1731       $M_CLS_1
 0B87:17C2       $M_CLS_2
 0B87:17E7       $M_MSGSERV_1
 0B87:1808       $M_MSGSERV_2
 0B87:0F9E       amis_sign
 0B87:0EA8       CallParser
 0B87:1856       data_sysdispmsg
 0B87:189A       data_sysgetmsg
 0B87:1812       data_sysloadmsg
 0B51:0000       DOSBEEP
 0B51:005D       DOSEXIT
 0000:FE32  Abs  FIARQQ
 0000:0E32  Abs  FICRQQ
 0000:5C32  Abs  FIDRQQ
 0000:1632  Abs  FIERQQ
 0000:0632  Abs  FISRQQ
 0000:A23D  Abs  FIWRQQ
 0000:4000  Abs  FJARQQ
 0000:C000  Abs  FJCRQQ
 0000:8000  Abs  FJSRQQ
 0B87:3BCE       STKHQQ
 0B87:0650       SysParse
 0B59:0056       VIOSCROLLUP
 0B59:0009       VIOSETCURPOS
 0B59:00C3       VIOWRTCHARSTRATT
 0000:733E       _atof
 0B87:3B1E       _BAD_BLOCK_part
 0B87:5346       _boot_record
 0000:7198       _brkctl
 0000:1B04       _change_active_partition
 0000:5854       _check_disk_validity
 0000:5CE9       _check_format
 0000:1F39       _check_valid_environment
 0000:5B8C       _check_yn_input
 0000:4590       _clear_screen
 0000:0FE8       _create_partition
 0B87:5548       _cur_disk
 0B87:4EB1       _cur_disk_buff
 0000:5A36       _cylinders_to_mbytes
 0000:5AB0       _cylinders_to_percent
 0B87:3B10       _debug_msg
 0000:04FC       _delete_partition
 0000:4EEA       _DiskIo
 0B87:596C       _disk_access
 0B87:4166       _disk_flag
 0000:28AA       _display
 0000:5550       _display_msg
 0B87:43BB       _display_page
 0000:1DE1       _display_partition_information
 0000:1EC7       _display_volume_information
 0000:1168       _dos_create_partition
 0000:06E8       _dos_delete
 0B87:3B18       _DOS_part
 0000:5B60       _dos_upper
 0000:0304       _do_main_menu
 0B87:4141       _dx_buff
 0B87:410A       _edata
 0B87:5980       _end
 0B87:3BBC       _environ
 0B87:3B95       _errno
 0B87:596A       _errorlevel
 0B87:3A88       _error_1
 0B87:3AAC       _error_10
 0B87:3AB0       _error_12
 0B87:3AB4       _error_13
 0B87:3AB8       _error_14
 0B87:3ABC       _error_15
 0B87:3AC0       _error_16
 0B87:3AC4       _error_17
 0B87:3AC8       _error_19
 0B87:3A8C       _error_2
 0B87:3ACC       _error_20
 0B87:3AD0       _error_21
 0B87:3AD4       _error_22
 0B87:3AD8       _error_23
 0B87:3ADC       _error_24
 0B87:3AE0       _error_25
 0B87:3AE4       _error_26
 0B87:3AE8       _error_27
 0B87:3AEC       _error_28
 0B87:3AF0       _error_29
 0B87:3A90       _error_3
 0B87:3AF4       _error_30
 0B87:3AF8       _error_31
 0B87:3AFC       _error_32
 0B87:3B00       _error_33
 0B87:3B04       _error_34
 0B87:3B08       _error_35
 0B87:3B0C       _error_36
 0B87:3A94       _error_4
 0B87:3A98       _error_5
 0B87:3A9C       _error_6
 0B87:3AA0       _error_7
 0B87:3AA4       _error_8
 0B87:3AA8       _error_9
 0000:5F10       _exit
 0B87:4E6C       _extended_buff
 0B87:4E77       _extended_flag
 0B87:3B1C       _EXTENDED_part
 0000:1526       _ext_create_partition
 0000:08D7       _ext_delete
 0B87:45C2       _ext_table
 0000:64F4       _fflush
 0000:438B       _find_active_partition
 0000:44D5       _find_ext_drive
 0000:3EBC       _find_ext_free_space
 0000:440B       _find_free_ext
 0000:42C6       _find_free_partition
 0000:444B       _find_logical_drive
 0000:43C9       _find_partition_location
 0000:4309       _find_partition_type
 0000:3A58       _find_part_free_space
 0000:4533       _find_previous_drive
 0000:6300       _flushall
 0000:6FDE       _free
 0B87:5556       _free_space
 0000:7494       _getch
 0000:7490       _getche
 0000:31F9       _get_alpha_input
 0000:32E9       _get_char_input
 0000:4A66       _get_disk_info
 0000:4E09       _get_drive_parameters
 0000:5BCD       _get_fs_and_vol
 0000:300A       _get_large_num_input
 0000:2DE8       _get_num_input
 0000:4489       _get_num_logical_dos_drives
 0000:4349       _get_partition_size
 0000:331C       _get_string_input
 0000:4697       _get_video_attribute
 0000:5C29       _get_volume_string
 0000:5589       _get_yes_no_values
 0000:2F08       _get_yn_input
 0B87:45C0       _good_disk
 0000:1F85       _init_partition_tables
 0000:45C0       _init_video_information
 0B87:4370       _input_col
 0B87:4378       _input_data
 0000:12EE       _input_dos_create
 0B87:45BC       _input_row
 0B87:4EB2       _insert
 0000:74AC       _int86
 0000:7580       _int86x
 0000:7614       _intdos
 0000:765C       _intdosx
 0B87:3B14       _internal_error
 0000:287B       _internal_program_error
 0000:73FE       _isatty
 0000:2387       _load_logical_drive
 0B87:5546       _logical_buff
 0B87:4E75       _logical_flag
 0000:6E2A       _lseek
 0000:0010       _main
 0000:46BE       _make_partition
 0000:48DB       _make_volume
 0000:6FF0       _malloc
 0B87:00E4       _master_boot_record
 0B87:416C       _max_head
 0B87:596B       _max_partition_size
 0B87:5344       _max_sector
 0000:593C       _mbytes_to_cylinders
 0000:770A       _memmove
 0000:7752       _memset
 0B87:39A0       _menu_1
 0B87:39C4       _menu_10
 0B87:39C8       _menu_11
 0B87:39CC       _menu_12
 0B87:39D0       _menu_13
 0B87:39D8       _menu_14
 0B87:39DC       _menu_15
 0B87:39E0       _menu_16
 0B87:39E8       _menu_17
 0B87:39F4       _menu_18
 0B87:39F8       _menu_19
 0B87:39A4       _menu_2
 0B87:3A00       _menu_20
 0B87:3A08       _menu_21
 0B87:3A0C       _menu_22
 0B87:3A14       _menu_23
 0B87:3A18       _menu_24
 0B87:3A1C       _menu_25
 0B87:3A20       _menu_26
 0B87:3A24       _menu_27
 0B87:3A28       _menu_28
 0B87:3A2C       _menu_29
 0B87:39A8       _menu_3
 0B87:3A30       _menu_30
 0B87:3A34       _menu_31
 0B87:3A38       _menu_32
 0B87:3A3C       _menu_33
 0B87:3A40       _menu_34
 0B87:3A48       _menu_35
 0B87:3A4C       _menu_36
 0B87:3A50       _menu_37
 0B87:3A54       _menu_38
 0B87:39E4       _menu_39
 0B87:39AC       _menu_4
 0B87:3A10       _menu_40
 0B87:3A44       _menu_41
 0B87:39EC       _menu_42
 0B87:39FC       _menu_43
 0B87:3A04       _menu_44
 0B87:39D4       _menu_45
 0B87:39F0       _menu_46
 0B87:39B0       _menu_5
 0B87:39B4       _menu_6
 0B87:39B8       _menu_7
 0B87:39BC       _menu_8
 0B87:39C0       _menu_9
 0B87:4E62       _mono_flag
 0B87:43BA       _next_letter
 0B87:4372       _No
 0B87:3B22       _NON_DOS_part
 0B87:0584       _NOVAL
 0B87:4EA7       _no_fatal_error
 0000:2C0A       _number_in_msg
 0B87:4E76       _number_of_drives
 0000:5D44       _parse
 0000:5624       _parse_command_line
 0000:571C       _parse_init
 0000:58B7       _Parse_msg
 0B87:5554       _Parse_Ptr
 0B87:51D4       _part_table
 0B87:3B20       _PCIX_part
 0B87:4E74       _PercentFlag
 0000:2C4D       _percent_in_msg
 0000:5B21       _percent_to_cylinders
 0B87:0582       _pinsert
 0000:5518       _preload_messages
 0B87:4E72       _primary_buff
 0B87:43AC       _primary_flag
 0000:5867       _process_switch
 0000:76D0       _putch
 0B87:554A       _p_buff
 0B87:4EA8       _p_con
 0B87:4167       _p_p
 0B87:415C       _p_px
 0B87:4394       _p_swi1
 0B87:43AE       _p_swi2
 0B87:4E9C       _p_val
 0B87:45BE       _quiet_flag
 0000:4E58       _read_boot_record
 0000:2898       _reboot
 0B87:4140       _reboot_flag
 0000:2806       _reboot_system
 0B87:437A       _regs
 0B87:5966       _required_cyls
 0000:4638       _reset_video_information
 0000:76BA       _segread
 0B87:4E64       _segregs
 0000:77E6       _signal
 0B87:4E84       _sort
 0000:4232       _sort_ext_table
 0000:3DFE       _sort_part_table
 0000:752A       _sprintf
 0B87:596E       _sp_buff
 0B87:4E78       _sp_val
 0000:6FCC       _stackavail
 0B87:3A58       _status_1
 0B87:3A7C       _status_10
 0B87:3A80       _status_11
 0B87:3A84       _status_12
 0B87:3A5C       _status_2
 0B87:3A60       _status_3
 0B87:3A64       _status_4
 0B87:3A68       _status_5
 0B87:3A6C       _status_6
 0B87:3A70       _status_7
 0B87:3A74       _status_8
 0B87:3A78       _status_9
 0000:725C       _strcat
 0000:76E0       _strchr
 0000:72CE       _strcmp
 0000:729C       _strcpy
 0000:2C90       _string_in_msg
 0000:72FA       _strlen
 0000:7316       _strncpy
 0B87:4388       _sublistp
 0000:5D88       _sysdispmsg
 0000:5D94       _sysgetmsg
 0000:5D8E       _sysloadmsg
 0000:3580       _table_display
 0000:3765       _table_drive_letter
 0B87:4E6E       _total_disk
 0B87:4374       _total_mbytes
 0000:73F4       _ultoa
 0B87:5552       _valid_input
 0000:4BD2       _verify_tracks
 0B87:51D2       _video_attribute
 0B87:415A       _video_mode
 0000:17D6       _volume_create
 0000:0A97       _volume_delete
 0000:37C0       _volume_display
 0000:2D27       _volume_in_msg
 0000:2FDC       _wait_for_ESC
 0000:6EA4       _write
 0000:4B38       _write_boot_record
 0000:523A       _write_ext_boot_to_disk
 0000:4F08       _write_info_to_disk
 0000:50B3       _write_master_boot_to_disk
 0B87:3B1A       _XENIX_part
 0B87:4E63       _Yes
 0B87:3B7A       __abrkp
 0B87:3B2A       __abrktb
 0B87:3B7A       __abrktbe
 0B87:3B7C       __acfinfo
 0000:9876  Abs  __acrtmsg
 0000:9876  Abs  __acrtused
 0B87:3BCC       __adbgmsg
 0B87:3B28       __aexit_rtn
 0B87:3B89       __aintdiv
 0000:7039       __amalloc
 0000:7178       __amallocbrk
 0B87:3D26       __amblksiz
 0000:711C       __amexpand
 0000:7156       __amlink
 0000:5E3D       __amsg_exit
 0000:7950       __aNlmul
 0000:7984       __aNlshl
 0000:7990       __aNNalmul
 0000:7990       __aNNaulmul
 0000:79B2       __aNuldiv
 0000:7950       __aNulmul
 0000:7A14       __aNulrem
 0000:7A80       __aNulshr
 0B87:3D20       __aseg1
 0B87:3D16       __asegds
 0B87:3D28       __asegh
 0B87:3D22       __asegn
 0B87:3D24       __asegr
 0B87:3B24       __asizds
 0B87:3D3A       __asizeC
 0B87:3D3B       __asizeD
 0000:5D9A       __astart
 0B87:3B26       __atopsp
 0B87:5766       __buferr
 0B87:43BC       __bufin
 0B87:4170       __bufout
 0000:8762       __cfltcvt
 0B87:3D2C       __cfltcvt_tab
 0B87:3BE6       __cflush
 0000:8446       __cftoe
 0000:8594       __cftof
 0000:86B0       __cftog
 0B87:3E3E       __chbuf
 0B87:3BC4       __child
 0000:5FE2       __chkstk
 0000:5E4C       __cinit
 0000:5E2E       __cintDIV
 0000:7780       __cltoasub
 0000:836E       __cropzeros
 0B87:3E40       __csigtab0
 0000:5F6C       __ctermsub
 0B87:3D3C       __ctype
 0B87:3D3C       __ctype_
 0000:778C       __cxtoa
 0000:7457       __DOSCREATECSALIAS
 0000:7422       __DOSDEVCONFIG
 0B87:3BA0       __doserrno
 0000:746D       __DOSFREESEG
 0000:7439       __DOSGETMACHINEMODE
 0000:62AC       __dosret0
 0000:62BF       __dosretax
 0000:62B4       __dosreturn
 0000:744E       __DOSSETVEC
 0B87:3B9D       __dosvermajor
 0B87:3B9E       __dosverminor
 0000:7476       __DOSWRITE
 0000:5F27       __exit
 0B87:3B8D       __fac
 0000:83F2       __fassign
 0000:5FBC       __FF_MSGBANNER
 0000:6332       __flsbuf
 0000:825B       __fltin
 0000:8234       __fltinf
 0000:829E       __fltout
 0000:9876  Abs  __fltused
 0000:8318       __forcdecpt
 087E:07D6       __fpemulator
 087E:0264       __FPEXCEPTION87
 0B87:3F3A       __fpinit
 087E:24BA       __FPINSTALL87
 087E:0024       __fpmath
 0000:7AA7       __fpsignal
 0B70:0164       __fptaskdata
 087E:24E9       __FPTERMINATE87
 0000:737E       __fptostr
 0000:5FDC       __fptrap
 0000:82E4       __ftol
 0000:6488       __getbuf
 0B87:3BC7       __intno
 0B87:3BE8       __iob
 0B87:3C88       __iob2
 0B87:3D00       __lastiob
 0000:62CC       __maperror
 0000:626A       __myalloc
 0B87:3BA2       __nfile
 0000:6FDE       __nfree
 0000:6FF0       __nmalloc
 0000:6216       __NMSG_TEXT
 0000:6241       __NMSG_WRITE
 0000:5FF8       __nullcheck
 0B87:3BA0       __oserr
 0B87:3BA4       __osfile
 0B87:3B9D       __osmajor
 0B87:3B9E       __osminor
 0B87:3B9F       __osmode
 0B87:3B9D       __osversion
 0000:6562       __output
 0B87:3BC6       __ovlflag
 0B87:3BC8       __ovlvec
 0B87:3BBE       __pgmptr
 0000:83C4       __positive
 0B87:3B9B       __psp
 0B87:3B99       __pspadr
 0B87:3D28       __QChdata
 0000:601A       __setargv
 0000:61A8       __setenvp
 0000:787D       __sigentry
 0B87:3D38       __sigintoff
 0B87:3D36       __sigintseg
 0B87:3B97       __umaskval
 0000:7940       __wrt2err
 0B87:3BB8       ___argc
 0B87:3BBA       ___argv

  Address         Publics by Value

 0000:0010       _main
 0000:0304       _do_main_menu
 0000:04FC       _delete_partition
 0000:0632  Abs  FISRQQ
 0000:06E8       _dos_delete
 0000:08D7       _ext_delete
 0000:0A97       _volume_delete
 0000:0E32  Abs  FICRQQ
 0000:0FE8       _create_partition
 0000:1168       _dos_create_partition
 0000:12EE       _input_dos_create
 0000:1526       _ext_create_partition
 0000:1632  Abs  FIERQQ
 0000:17D6       _volume_create
 0000:1B04       _change_active_partition
 0000:1DE1       _display_partition_information
 0000:1EC7       _display_volume_information
 0000:1F39       _check_valid_environment
 0000:1F85       _init_partition_tables
 0000:2387       _load_logical_drive
 0000:2806       _reboot_system
 0000:287B       _internal_program_error
 0000:2898       _reboot
 0000:28AA       _display
 0000:2C0A       _number_in_msg
 0000:2C4D       _percent_in_msg
 0000:2C90       _string_in_msg
 0000:2D27       _volume_in_msg
 0000:2DE8       _get_num_input
 0000:2F08       _get_yn_input
 0000:2FDC       _wait_for_ESC
 0000:300A       _get_large_num_input
 0000:31F9       _get_alpha_input
 0000:32E9       _get_char_input
 0000:331C       _get_string_input
 0000:3580       _table_display
 0000:3765       _table_drive_letter
 0000:37C0       _volume_display
 0000:3A58       _find_part_free_space
 0000:3DFE       _sort_part_table
 0000:3EBC       _find_ext_free_space
 0000:4000  Abs  FJARQQ
 0000:4232       _sort_ext_table
 0000:42C6       _find_free_partition
 0000:4309       _find_partition_type
 0000:4349       _get_partition_size
 0000:438B       _find_active_partition
 0000:43C9       _find_partition_location
 0000:440B       _find_free_ext
 0000:444B       _find_logical_drive
 0000:4489       _get_num_logical_dos_drives
 0000:44D5       _find_ext_drive
 0000:4533       _find_previous_drive
 0000:4590       _clear_screen
 0000:45C0       _init_video_information
 0000:4638       _reset_video_information
 0000:4697       _get_video_attribute
 0000:46BE       _make_partition
 0000:48DB       _make_volume
 0000:4A66       _get_disk_info
 0000:4B38       _write_boot_record
 0000:4BD2       _verify_tracks
 0000:4E09       _get_drive_parameters
 0000:4E58       _read_boot_record
 0000:4EEA       _DiskIo
 0000:4F08       _write_info_to_disk
 0000:50B3       _write_master_boot_to_disk
 0000:523A       _write_ext_boot_to_disk
 0000:5518       _preload_messages
 0000:5550       _display_msg
 0000:5589       _get_yes_no_values
 0000:5624       _parse_command_line
 0000:571C       _parse_init
 0000:5854       _check_disk_validity
 0000:5867       _process_switch
 0000:58B7       _Parse_msg
 0000:593C       _mbytes_to_cylinders
 0000:5A36       _cylinders_to_mbytes
 0000:5AB0       _cylinders_to_percent
 0000:5B21       _percent_to_cylinders
 0000:5B60       _dos_upper
 0000:5B8C       _check_yn_input
 0000:5BCD       _get_fs_and_vol
 0000:5C29       _get_volume_string
 0000:5C32  Abs  FIDRQQ
 0000:5CE9       _check_format
 0000:5D44       _parse
 0000:5D88       _sysdispmsg
 0000:5D8E       _sysloadmsg
 0000:5D94       _sysgetmsg
 0000:5D9A       __astart
 0000:5E2E       __cintDIV
 0000:5E3D       __amsg_exit
 0000:5E4C       __cinit
 0000:5F10       _exit
 0000:5F27       __exit
 0000:5F6C       __ctermsub
 0000:5FBC       __FF_MSGBANNER
 0000:5FDC       __fptrap
 0000:5FE2       __chkstk
 0000:5FF8       __nullcheck
 0000:601A       __setargv
 0000:61A8       __setenvp
 0000:6216       __NMSG_TEXT
 0000:6241       __NMSG_WRITE
 0000:626A       __myalloc
 0000:62AC       __dosret0
 0000:62B4       __dosreturn
 0000:62BF       __dosretax
 0000:62CC       __maperror
 0000:6300       _flushall
 0000:6332       __flsbuf
 0000:6488       __getbuf
 0000:64F4       _fflush
 0000:6562       __output
 0000:6E2A       _lseek
 0000:6EA4       _write
 0000:6FCC       _stackavail
 0000:6FDE       __nfree
 0000:6FDE       _free
 0000:6FF0       _malloc
 0000:6FF0       __nmalloc
 0000:7039       __amalloc
 0000:711C       __amexpand
 0000:7156       __amlink
 0000:7178       __amallocbrk
 0000:7198       _brkctl
 0000:725C       _strcat
 0000:729C       _strcpy
 0000:72CE       _strcmp
 0000:72FA       _strlen
 0000:7316       _strncpy
 0000:733E       _atof
 0000:737E       __fptostr
 0000:73F4       _ultoa
 0000:73FE       _isatty
 0000:7422       __DOSDEVCONFIG
 0000:7439       __DOSGETMACHINEMODE
 0000:744E       __DOSSETVEC
 0000:7457       __DOSCREATECSALIAS
 0000:746D       __DOSFREESEG
 0000:7476       __DOSWRITE
 0000:7490       _getche
 0000:7494       _getch
 0000:74AC       _int86
 0000:752A       _sprintf
 0000:7580       _int86x
 0000:7614       _intdos
 0000:765C       _intdosx
 0000:76BA       _segread
 0000:76D0       _putch
 0000:76E0       _strchr
 0000:770A       _memmove
 0000:7752       _memset
 0000:7780       __cltoasub
 0000:778C       __cxtoa
 0000:77E6       _signal
 0000:787D       __sigentry
 0000:7940       __wrt2err
 0000:7950       __aNulmul
 0000:7950       __aNlmul
 0000:7984       __aNlshl
 0000:7990       __aNNalmul
 0000:7990       __aNNaulmul
 0000:79B2       __aNuldiv
 0000:7A14       __aNulrem
 0000:7A80       __aNulshr
 0000:7AA7       __fpsignal
 0000:7AE1       $i8_input
 0000:7F35       $i8_output
 0000:8000  Abs  FJSRQQ
 0000:81F6       $i8_tpwr10
 0000:8234       __fltinf
 0000:825B       __fltin
 0000:829E       __fltout
 0000:82E4       __ftol
 0000:8318       __forcdecpt
 0000:836E       __cropzeros
 0000:83C4       __positive
 0000:83F2       __fassign
 0000:8446       __cftoe
 0000:8594       __cftof
 0000:86B0       __cftog
 0000:8762       __cfltcvt
 087E:0024       __fpmath
 087E:0264       __FPEXCEPTION87
 087E:07D6       __fpemulator
 0000:9876  Abs  __acrtused
 0000:9876  Abs  __acrtmsg
 0000:9876  Abs  __fltused
 0000:A23D  Abs  FIWRQQ
 087E:24BA       __FPINSTALL87
 087E:24E9       __FPTERMINATE87
 0B51:0000       DOSBEEP
 0B51:005D       DOSEXIT
 0B59:0009       VIOSETCURPOS
 0B59:0056       VIOSCROLLUP
 0B59:00C3       VIOWRTCHARSTRATT
 0B70:0164       __fptaskdata
 0B87:00E4       _master_boot_record
 0B87:0582       _pinsert
 0B87:0584       _NOVAL
 0B87:0650       SysParse
 0000:C000  Abs  FJCRQQ
 0B87:0EA8       CallParser
 0B87:0F9E       amis_sign
 0B87:1731       $M_CLS_1
 0B87:17C2       $M_CLS_2
 0B87:17E7       $M_MSGSERV_1
 0B87:1808       $M_MSGSERV_2
 0B87:1812       data_sysloadmsg
 0B87:1856       data_sysdispmsg
 0B87:189A       data_sysgetmsg
 0B87:39A0       _menu_1
 0B87:39A4       _menu_2
 0B87:39A8       _menu_3
 0B87:39AC       _menu_4
 0B87:39B0       _menu_5
 0B87:39B4       _menu_6
 0B87:39B8       _menu_7
 0B87:39BC       _menu_8
 0B87:39C0       _menu_9
 0B87:39C4       _menu_10
 0B87:39C8       _menu_11
 0B87:39CC       _menu_12
 0B87:39D0       _menu_13
 0B87:39D4       _menu_45
 0B87:39D8       _menu_14
 0B87:39DC       _menu_15
 0B87:39E0       _menu_16
 0B87:39E4       _menu_39
 0B87:39E8       _menu_17
 0B87:39EC       _menu_42
 0B87:39F0       _menu_46
 0B87:39F4       _menu_18
 0B87:39F8       _menu_19
 0B87:39FC       _menu_43
 0B87:3A00       _menu_20
 0B87:3A04       _menu_44
 0B87:3A08       _menu_21
 0B87:3A0C       _menu_22
 0B87:3A10       _menu_40
 0B87:3A14       _menu_23
 0B87:3A18       _menu_24
 0B87:3A1C       _menu_25
 0B87:3A20       _menu_26
 0B87:3A24       _menu_27
 0B87:3A28       _menu_28
 0B87:3A2C       _menu_29
 0B87:3A30       _menu_30
 0B87:3A34       _menu_31
 0B87:3A38       _menu_32
 0B87:3A3C       _menu_33
 0B87:3A40       _menu_34
 0B87:3A44       _menu_41
 0B87:3A48       _menu_35
 0B87:3A4C       _menu_36
 0B87:3A50       _menu_37
 0B87:3A54       _menu_38
 0B87:3A58       _status_1
 0B87:3A5C       _status_2
 0B87:3A60       _status_3
 0B87:3A64       _status_4
 0B87:3A68       _status_5
 0B87:3A6C       _status_6
 0B87:3A70       _status_7
 0B87:3A74       _status_8
 0B87:3A78       _status_9
 0B87:3A7C       _status_10
 0B87:3A80       _status_11
 0B87:3A84       _status_12
 0B87:3A88       _error_1
 0B87:3A8C       _error_2
 0B87:3A90       _error_3
 0B87:3A94       _error_4
 0B87:3A98       _error_5
 0B87:3A9C       _error_6
 0B87:3AA0       _error_7
 0B87:3AA4       _error_8
 0B87:3AA8       _error_9
 0B87:3AAC       _error_10
 0B87:3AB0       _error_12
 0B87:3AB4       _error_13
 0B87:3AB8       _error_14
 0B87:3ABC       _error_15
 0B87:3AC0       _error_16
 0B87:3AC4       _error_17
 0B87:3AC8       _error_19
 0B87:3ACC       _error_20
 0B87:3AD0       _error_21
 0B87:3AD4       _error_22
 0B87:3AD8       _error_23
 0B87:3ADC       _error_24
 0B87:3AE0       _error_25
 0B87:3AE4       _error_26
 0B87:3AE8       _error_27
 0B87:3AEC       _error_28
 0B87:3AF0       _error_29
 0B87:3AF4       _error_30
 0B87:3AF8       _error_31
 0B87:3AFC       _error_32
 0B87:3B00       _error_33
 0B87:3B04       _error_34
 0B87:3B08       _error_35
 0B87:3B0C       _error_36
 0B87:3B10       _debug_msg
 0B87:3B14       _internal_error
 0B87:3B18       _DOS_part
 0B87:3B1A       _XENIX_part
 0B87:3B1C       _EXTENDED_part
 0B87:3B1E       _BAD_BLOCK_part
 0B87:3B20       _PCIX_part
 0B87:3B22       _NON_DOS_part
 0B87:3B24       __asizds
 0B87:3B26       __atopsp
 0B87:3B28       __aexit_rtn
 0B87:3B2A       __abrktb
 0B87:3B7A       __abrktbe
 0B87:3B7A       __abrkp
 0B87:3B7C       __acfinfo
 0B87:3B89       __aintdiv
 0B87:3B8D       __fac
 0B87:3B95       _errno
 0B87:3B97       __umaskval
 0B87:3B99       __pspadr
 0B87:3B9B       __psp
 0B87:3B9D       __dosvermajor
 0B87:3B9D       __osmajor
 0B87:3B9D       __osversion
 0B87:3B9E       __dosverminor
 0B87:3B9E       __osminor
 0B87:3B9F       __osmode
 0B87:3BA0       __oserr
 0B87:3BA0       __doserrno
 0B87:3BA2       __nfile
 0B87:3BA4       __osfile
 0B87:3BB8       ___argc
 0B87:3BBA       ___argv
 0B87:3BBC       _environ
 0B87:3BBE       __pgmptr
 0B87:3BC4       __child
 0B87:3BC6       __ovlflag
 0B87:3BC7       __intno
 0B87:3BC8       __ovlvec
 0B87:3BCC       __adbgmsg
 0B87:3BCE       STKHQQ
 0B87:3BE6       __cflush
 0B87:3BE8       __iob
 0B87:3C88       __iob2
 0B87:3D00       __lastiob
 0B87:3D16       __asegds
 0B87:3D20       __aseg1
 0B87:3D22       __asegn
 0B87:3D24       __asegr
 0B87:3D26       __amblksiz
 0B87:3D28       __asegh
 0B87:3D28       __QChdata
 0B87:3D2C       __cfltcvt_tab
 0B87:3D36       __sigintseg
 0B87:3D38       __sigintoff
 0B87:3D3A       __asizeC
 0B87:3D3B       __asizeD
 0B87:3D3C       __ctype_
 0B87:3D3C       __ctype
 0B87:3E3E       __chbuf
 0B87:3E40       __csigtab0
 0B87:3E8E       $i8_inpbas
 0B87:3E8F       $i8_input_ws
 0B87:3E90       $i8_implicit_exp
 0B87:3F3A       __fpinit
 0B87:410A       _edata
 0B87:4140       _reboot_flag
 0B87:4141       _dx_buff
 0B87:415A       _video_mode
 0B87:415C       _p_px
 0B87:4166       _disk_flag
 0B87:4167       _p_p
 0B87:416C       _max_head
 0B87:4170       __bufout
 0B87:4370       _input_col
 0B87:4372       _No
 0B87:4374       _total_mbytes
 0B87:4378       _input_data
 0B87:437A       _regs
 0B87:4388       _sublistp
 0B87:4394       _p_swi1
 0B87:43AC       _primary_flag
 0B87:43AE       _p_swi2
 0B87:43BA       _next_letter
 0B87:43BB       _display_page
 0B87:43BC       __bufin
 0B87:45BC       _input_row
 0B87:45BE       _quiet_flag
 0B87:45C0       _good_disk
 0000:FE32  Abs  FIARQQ
 0B87:45C2       _ext_table
 0B87:4E62       _mono_flag
 0B87:4E63       _Yes
 0B87:4E64       _segregs
 0B87:4E6C       _extended_buff
 0B87:4E6E       _total_disk
 0B87:4E72       _primary_buff
 0B87:4E74       _PercentFlag
 0B87:4E75       _logical_flag
 0B87:4E76       _number_of_drives
 0B87:4E77       _extended_flag
 0B87:4E78       _sp_val
 0B87:4E84       _sort
 0B87:4E9C       _p_val
 0B87:4EA7       _no_fatal_error
 0B87:4EA8       _p_con
 0B87:4EB1       _cur_disk_buff
 0B87:4EB2       _insert
 0B87:51D2       _video_attribute
 0B87:51D4       _part_table
 0B87:5344       _max_sector
 0B87:5346       _boot_record
 0B87:5546       _logical_buff
 0B87:5548       _cur_disk
 0B87:554A       _p_buff
 0B87:5552       _valid_input
 0B87:5554       _Parse_Ptr
 0B87:5556       _free_space
 0B87:5766       __buferr
 0B87:5966       _required_cyls
 0B87:596A       _errorlevel
 0B87:596B       _max_partition_size
 0B87:596C       _disk_access
 0B87:596E       _sp_buff
 0B87:5980       _end

Program entry point at 0000:5D9A
